:020000040000FA
:020000002228B4
:0800080018201E089500452098
:100010001E08F000422017129712701B1716F01BD3
:1000200097160B118C108B17452002308C0009009D
:10003000452014309B00422061309F001F151F197E
:100040001F28080042208615043092009501960171
:100050007D3095000C309700452007309C00003023
:100060009B0010309F0007308100FA309200F03082
:100070008600C0308B0002308C00000000000000C1
:1000800000003D28031383120800031383160800A1
:0C009000031783120800031783160800F2
:02400E00422F3F
:02401000FC3F73
:00000001FF
